:020000040000FA
:020000000A28CC
:020008000E28C0
:0C0014004B30CB0040200D280E28CC0003
:10002000CB034B0884004C0880000800CC004B0830
:1000300084000008CE00CB0A4C080800CC004E0813
:1000400084004C08800008008400000808004E0668
:10005000CE064E060800CC004B0884004C08000673
:0600600080060006080006
:100080001F306500003066002030860001300F20F0
:100090000921CB0A0030A7000030A2000030A100E7
:1000A0000130003E0319F828F920A00020080F2095
:1000B000103016204E05003E0319E2280030A7003C
:1000C00021080F20003016203621003E0319E128B8
:1000D00020080F200F3016204E05A00020080F200A
:1000E0000C3016203621003E0319B32822080F20B9
:1000F000043016203621003E0319832823080F20E0
:100100000230162036215221003E03198C28240883
:100110000F200430162036215221003E0319952865
:1001200025080F200830162036215221003E0319E1
:100130009E2826080F200630162036215221003E28
:100140000319AA2810300F20FB20CB0A02300F2001
:100150000921CB0A00300F20FB20CB0A0030A2007F
:100160000030A100E128A20A0130A10022080F20DE
:10017000013016203621003E0319C1282008A300B3
:10018000E12822080F20023016203621003E0319F4
:10019000CC282008A400E12822080F2003301620D4
:1001A0003621003E0319D7282008A500E12822089F
:1001B0000F20043016203621003E0319E1282008C4
:1001C000A600F3280030A100A70A27080F201E3040
:1001D00016204821003E0319F3280030A200003009
:1001E0000F20FB20CB0A64300F200021CB0A5028BF
:1001F0000800050808004B08840000088600080075
:100200004B082420CF00CC01CC0B0429CF0B0429B0
:100210000800CB034B080F20003016201E204B088F
:1002200024200F2002304B07242016203E21003EC0
:10023000031D232934294B080F202420013E1620BA
:100240001E20FF3E0F29FA300F200021CB0AFA3082
:100250000F200021CB0AFA300F200021CB0AFA3000
:100260000F200021CB0A1B29CB0A08004E060319D8
:10027000013400344E06031D013400344E020318CD
:100280000034031D013400344E02031800340134DD
:100290004E02031C003401344E02031801340319CA
:0C02A00001340034003803190800013458
:02400E00F23F7F
:00000001FF
